:1000000000308A00532A00003A30840000080319A7
:1000100016280630F800F701F70B0C28F80B0B2810
:100020007B30F700F70B1228800B092800341030C2
:10003000F700FA01C601C30CC20C031C25284408B2
:10004000FA070318C60A4508C607C60CFA0CF90CCD
:10005000F80CF70B1B280034F801F901F701FA013D
:100060004908031D36284808031950281030CA00D3
:100070000310C60DC70DF70DFA0D49087A02031DCE
:10008000432848087702031C4C284808F702031C41
:10009000FA034908FA020314F80DF90DCA0B3828BF
:1000A00000008A1182284108A3004008A2003F08EE
:1000B000A1003E08A0003B08A5003A08A4003D08A6
:1000C000A7003C08A6003B08C3003A08C2003B0852
:1000D000C5003A08C40017207908C3007808C20098
:1000E00003103C0DF9003D0DFA007908C4007A08B0
:1000F000C5004308C7007808C6007A08C900790817
:10010000C8002C2878083E02B0003F08B1007908EA
:10011000031C790FB1024008B2000030031C01300B
:10012000B2024108B3000030031C0130B3023908A9
:10013000B40000343408FC3E03185A29043E5C29FC
:100140005A292308AD002208AC002108AB00200882
:10015000AA005A292408AA0725080318250FAB0767
:10016000003003180130AC07003003180130AD0730
:100170005A2933082D02031CD628031DCF28320824
:100180002C02031CD628031DCF2831082B02031C88
:10019000D628031DCF2830082A02031CD62826089B
:1001A000AE022708031C270FAF020229AF1FDB286E
:1001B000A51FE728DD28A51B02292F082502031CFF
:1001C0000229031DE72824082E0203180229260805
:1001D000AE070318AF0A2708AF07A51FF228AF1F05
:1001E000FE28F428AF1B022925082F02031C022930
:1001F000031DFE282E082402031802292508AF003B
:100200002408AE0026082A07B9002B08BA002708E0
:100210000318270FBA072C08BB0000300318013061
:10022000BB072D08BC00003003180130BC072308B1
:100230003C02031C2D29031D2F2922083B02031C0D
:100240002D29031D2F2921083A02031C2D29031DE6
:100250002F292008390203182F29AF1F3A29230814
:10026000AD002208AC002108AB002008AA00AF01B5
:10027000AE01B4012E08F7002F08F800F901FA01C9
:10028000AF1F4429F903FA032A08F7072B080318BC
:100290002B0FF8072C0803182C0FF9072D0803184B
:1002A0002D0FFA077A08AD007908AC007808AB008A
:1002B0007708AA008A1175290A148A100A11820780
:1002C000A028B928A128AA280330BE02031C72293D
:1002D0003E308400000803197229702900000000D4
:1002E000800B6E298A1181299A28B901BA01BB01B4
:1002F000BC019701970186110230BD00F730BE00A6
:100300006429BD0B7E290030F8001F08C739780426
:100310009F001030F700F70B8B2900001F151F19E5
:100320008F291E08BA01B9000830F8001F08C73924
:1003300078049F001030F700F70B9C2900001F1570
:100340001F19A0291E08BC01BB00861506100C3021
:1003500097003B083902F7003A08FA003C08031CF2
:100360003C0FFA027708A8070318A90A7A08A90718
:10037000B4080319192A2808F7002908F800F90118
:10038000FA01A91FC529F903FA0377082A02F70021
:100390007808031C780FCE292B08CF292B02F800F0
:1003A0007908031C790FD6292C08D7292C02F900CB
:1003B0007A08031C7A0FDE292D08DF292D02FA00A6
:1003C0007808BC007708BB00C3010330C2003C08BA
:1003D000C5003B08C40017207908BE007808BD009E
:1003E00037083B02F7003C08FA003808031C380FB6
:1003F000FA027708BF007A08C000C3010A30C200C1
:100400007A08C5007708C400172078083D07B900AE
:100410003E08BA000318BA0A7908BA073B08B507BC
:100420000318B60A3C08B6073C08B8003B08B700FA
:100430001B2ABA01B9013A08BE003908BD00BE1F27
:10044000242A05118515262A851105153E08FA006E
:100450003D08BE1F342A3D08003CF700FA013E0863
:10046000031C3E0FFA027708BF007A08C00040085C
:10047000033C03183F2A0330C000FF30BF00400890
:10048000F9003F08F800F90CF80CF90CF80CF90C1D
:1004900078089500F90C790C3039F7001708CF3936
:1004A00077049700003484011F30830583161F12E0
:1004B0009F121B0880390F389B00073083129F0062
:1004C00040308316990026309800903083129800AF
:1004D000A801A901AA01AB01AC01AD01AE01AF01B8
:1004E000B401B501B601B701B801073083169C000D
:1004F00005081030F700F70B7B2A00001C08831258
:100500000D1383169D01F3306500D43066001F1271
:100510009F121B08803903389B001F1383121F177B
:100520009F1783169F1383121F140030F8001F08B3
:10053000C73978049F0006100C3097000030F8008F
:1005400005389200FF308316920083129501051141
:1005500085110430B900FA30BA000420B90BAB2A77
:100560000130B900BB017830BA00BD010130BC00D8
:10057000C101C0019C30BF004030BE005320B40810
:100580000319C72A0530BA0004207421BF2A02309B
:10059000B900BB01BA01BD01BC01C101C0019C3061
:1005A000BF004030BE0053200530BA000420742143
:0405B000D42A6300E6
:04400E002A3FFC3F0A
:00000001FF
